:020000040000FA
:0408000072EF06F09D
:1008100003B207EF05F0F2B422EF05F09EB02AEF25
:1008200005F09EB232EF05F0F2A81AEF04F0F2B232
:100830001CEF04F050EF06F0CD90F2929EA026EF50
:1008400004F00101463F26EF04F0472BA1C1A5F1BA
:10085000A2C1A6F1A3C1A7F1A4C1A8F19DC1A1F1B4
:100860009EC1A2F19FC1A3F1A0C1A4F199C19DF1C4
:100870009AC19EF19BC19FF19CC1A0F195C199F1D4
:1008800096C19AF197C19BF198C19CF191C195F1E4
:1008900092C196F193C197F194C198F18DC191F1F4
:1008A0008EC192F18FC193F190C194F189C18DF104
:1008B0008AC18EF18BC18FF18CC190F1CECF89F1BD
:1008C000CFCF8AF146C18BF147C18CF1CF6ACE6A96
:1008D0000101466B476B9E90CD800EBC0E8E0EBA0A
:1008E00075EF04F00E8A50EF06F00E8C0EBEB1EFDD
:1008F00004F089C18DF18AC18EF18BC18FF18CC159
:1009000090F18DC191F18EC192F18FC193F190C19F
:1009100094F191C195F192C196F193C197F194C16F
:1009200098F195C199F196C19AF197C19BF198C13F
:100930009CF199C19DF19AC19EF19BC19FF19CC10F
:10094000A0F19DC1A1F19EC1A2F19FC1A3F1A0C1DF
:10095000A4F1A1C1A5F1A2C1A6F1A3C1A7F1A4C1AF
:10096000A8F10101516B526B536B546B89515127A4
:100970008A5152238B5153238C5154238D5151272B
:100980008E5152238F51532390515423915151270B
:1009900092515223935153239451542395515127EB
:1009A00096515223975153239851542399515127CB
:1009B0009A5152239B5153239C5154239D515127AB
:1009C0009E5152239F515323A0515423A15151278B
:1009D000A2515223A3515323A4515423A55151276B
:1009E000A6515223A7515323A8515423D8905433CE
:1009F000533352335133D8905433533352335133EA
:100A0000D890543353335233513350EF06F003929E
:100A1000030103EE00F080517F0BE92604C0EFFFD5
:100A2000802B8151805D700BD8A48B820000805197
:100A3000815D700BD8A48B9281518019D8B4079036
:100A400050EF06F0F2940101383F50EF06F0392BD9
:100A500050EF06F09E900101463F50EF06F0472B05
:100A600050EF06F09E92C3CF48F1C4CF49F1C28245
:100A700007B49DEF05F03AC13EF13BC13FF13CC1E7
:100A800040F13DC141F151C155F152C156F153C13F
:100A900057F154C158F189C1A9F18AC1AAF18BC19A
:100AA000ABF18CC1ACF18DC1ADF18EC1AEF18FC196
:100AB000AFF190C1B0F191C1B1F192C1B2F193C166
:100AC000B3F194C1B4F195C1B5F196C1B6F197C136
:100AD000B7F198C1B8F199C1B9F19AC1BAF19BC106
:100AE000BBF19CC1BCF19DC1BDF19EC1BEF19FC1D6
:100AF000BFF1A0C1C0F1A1C1C1F1A2C1C2F1A3C1A6
:100B0000C3F1A4C1C4F1A5C1C5F1A6C1C6F1A7C175
:100B1000C7F1A8C1C8F1010148514E2749514F23DF
:100B2000E86A50230D2E9DEF05F04FC14AF150C1E8
:100B30004BF14E6B4F6B506B078E0201002F50EF45
:100B400006F03C0E006F01017D67AEEF05F07E6799
:100B5000AEEF05F07F67AEEF05F08067B2EF05F00E
:100B6000E2EF05F081C100F182C101F183C102F120
:100B700084C103F10101010E046F000E056F000E28
:100B8000066F000E076FF1EC13F000C181F101C197
:100B900082F102C183F103C184F10067D7EF05F050
:100BA0000167D7EF05F00267D7EF05F00367E2EFC3
:100BB00005F07DC181F17EC182F17FC183F180C1E9
:100BC00084F10E80D57ED5BE69D0D6CF3AF1D7CF8D
:100BD0003BF138C13CF1E86AE8CF3DF10F903AC1F2
:100BE00000F13BC101F13CC102F13DC103F1010142
:100BF0000A0E046F000E056F000E066F000E076FE1
:100C0000F1EC13F000AF0F80010147A714EF06F0DD
:100C10000E9A0E9C0E9E0101000E516F600E526FD7
:100C20003D0E536F080E546F01013ABF24EF06F0DA
:100C30003B6724EF06F03C6724EF06F03D6724EFA6
:100C400006F0F28849EF06F0F298516B526B536B45
:100C5000546B896B8A6B8B6B8C6B8D6B8E6B8F6B14
:100C6000906B916B926B936B946B956B966B976B90
:100C7000986B996B9A6B9B6B9C6B9D6B9E6B9F6B40
:100C8000A06BA16BA26BA36BA46BA56BA66BA76BF0
:100C9000A86BD76AD66A0101386B396B50EF06F042
:100CA00002C0E0FF005001C0D8FF1000A6B256EF0E
:100CB00006F00CC0A9FF0BC0A8FFA69EA69CA684A8
:100CC000F29E550EA76EAA0EA76EA682F28EA6946D
:100CD000A6B268EF06F01200A96EA69EA69CA6809A
:100CE000A8501200076A0E6A0F6A0F010E0EC16E3D
:100CF000860EC06E030EC26E0F01896A110E926ECF
:100D0000080E8A6EF10E936E8B6A800E946EF18ED1
:100D10000D6A01014E6B4F6B506B4A6B4B6BF29A35
:100D200001013A6B3B6B3C6B3D6B3E6B3F6B406B29
:100D3000416B426B436B446B456B386B396BD76AC5
:100D4000D66A0F01280ED56EF28A9D90B00ECD6E38
:100D50000101516B526B536B546B556B566B576B58
:100D6000586B596B5A6B5B6B5C6B466B476BCF6A0E
:100D7000CE6A0E9A0E9C0E9E9D80760ECA6E9D8245
:100D800002013C0E006FCC6A160E6CEC06F0E8CF48
:100D900000F1170E6CEC06F0E8CF01F1180E6CECC8
:100DA00006F0E8CF02F1190E6CEC06F0E8CF03F183
:100DB000010103AFF6EF06F0E8EC14F0160E0C6E2E
:100DC00000C10BF056EC06F0170E0C6E01C10BF0D3
:100DD00056EC06F0180E0C6E02C10BF056EC06F045
:100DE000190E0C6E03C10BF056EC06F000C17DF13C
:100DF00001C17EF102C17FF103C180F100C181F127
:100E000001C182F102C183F103C184F11A0E6CECBD
:100E100006F0E8CF00F11B0E6CEC06F0E8CF01F114
:100E20001C0E6CEC06F0E8CF02F11D0E6CEC06F027
:100E3000E8CF03F1010103AF4CEF07F0E8EC14F049
:100E40001A0E0C6E00C10BF056EC06F01B0E0C6E69
:100E500001C10BF056EC06F01C0E0C6E02C10BF03B
:100E600056EC06F01D0E0C6E03C10BF056EC06F0AE
:100E70001A0E6CEC06F0E8CF00F11B0E6CEC06F0DD
:100E8000E8CF01F11C0E6CEC06F0E8CF02F11D0E6C
:100E90006CEC06F0E8CF03F100C185F101C186F1E9
:100EA00002C187F103C188F1240EAC6E900EAB6EC7
:100EB000240EAC6E080EB86E000EB06E1F0EAF6E34
:100EC0000401806B816B0F01900EAB6E0F019D8A48
:100ED0000301806B816BA26B8B9207900001F28EF5
:100EE000F28C07B0B5EF11F00EB096EF0CF00301E5
:100EF000805181197F0BD8B4B5EF11F013EE00F0DB
:100F000081517F0BE126812BE7CFE8FFE00BD8B4BE
:100F1000B5EF11F023EE82F0A2511F0BD926E7CFD7
:100F2000DFFFA22BDF50780AD8A4B5EF11F00780BD
:100F300081C100F182C101F183C102F184C103F1D9
:100F40000101040E046F000E056F000E066F000E07
:100F5000076FF1EC13F000AFB7EF07F00101030EDC
:100F6000816F000E826F000E836F000E846F03018D
:100F70008251720AD8B496EF0CF08251520AD8B45A
:100F800096EF0CF08251750AD8B496EF0CF08251AE
:100F9000630AD8B471EF0EF08251690AD8B451EFE8
:100FA00009F082517A0AD8B464EF0AF08251490AF2
:100FB000D8B4F0EF08F08251500AD8B40EEF08F020
:100FC0008251700AD8B451EF08F08251540AD8B453
:100FD0007CEF08F08251740AD8B4C2EF08F0825155
:100FE000730AD8B4C6EF0BF08251530AD8B42BEF72
:100FF0000CF0A6EF0EF0040114EE00F080517F0B10
:10100000E12682C4E7FF802B12000D0E826FFBECFD
:1010100007F00A0E826FFBEC07F0120083C31EF18B
:1010200084C31FF185C320F186C321F187C322F158
:1010300088C323F189C324F18AC325F18BC326F128
:101040008CC327F1010136EC15F0ADEC14F0160E4F
:101050000C6E00C10BF056EC06F0170E0C6E01C1C1
:101060000BF056EC06F0180E0C6E02C10BF056ECAD
:1010700006F0190E0C6E03C10BF056EC06F000C121
:101080007DF101C17EF102C17FF103C180F100C198
:1010900081F101C182F102C183F103C184F1F0EF5A
:1010A00008F083C31EF184C31FF185C320F186C3FA
:1010B00021F187C322F188C323F189C324F18AC3B4
:1010C00025F18BC326F18CC327F1010136EC15F015
:1010D000ADEC14F000C17DF101C17EF102C17FF1E0
:1010E00003C180F100C181F101C182F102C183F12C
:1010F00003C184F1F0EF08F083C31EF184C31FF134
:1011000085C320F186C321F187C322F188C323F16F
:1011100089C324F18AC325F18CC326F18DC327F13D
:10112000010136EC15F0ADEC14F00101000E046F76
:10113000000E056F010E066F000E076F00EC14F035
:101140001A0E0C6E00C10BF056EC06F01B0E0C6E66
:1011500001C10BF056EC06F01C0E0C6E02C10BF038
:1011600056EC06F01D0E0C6E03C10BF056EC06F0AB
:1011700000C185F101C186F102C187F103C188F187
:10118000F0EF08F083C31EF184C31FF185C320F183
:1011900086C321F187C322F188C323F189C324F1D7
:1011A0008AC325F18CC326F18DC327F1010136ECEA
:1011B00015F0ADEC14F00101000E046F000E056F88
:1011C000010E066F000E076F00EC14F000C185F1F0
:1011D00001C186F102C187F103C188F1F0EF08F087
:1011E000160E6CEC06F0E8CF00F1170E6CEC06F072
:1011F000E8CF01F1180E6CEC06F0E8CF02F1190E01
:101200006CEC06F0E8CF03F18BEC14F0B7EC12F0C5
:101210000401730E826FFBEC07F004012C0E826F49
:10122000FBEC07F07DC100F17EC101F17FC102F14D
:1012300080C103F18BEC14F0B7EC12F00401730ED3
:10124000826FFBEC07F004012C0E826FFBEC07F0C1
:101250001A0E6CEC06F0E8CF00F11B0E6CEC06F0F9
:10126000E8CF01F11C0E6CEC06F0E8CF02F11D0E88
:101270006CEC06F0E8CF03F1C1EC0EF004012C0E8B
:10128000826FFBEC07F085C100F186C101F187C1D7
:1012900002F188C103F1C1EC0EF005EC08F0A6EFF5
:1012A0000EF00401690E826FFBEC07F004012C0EB6
:1012B000826FFBEC07F00101040E006F000E016F5E
:1012C000000E026F000E036F8BEC14F020C182F44D
:1012D0000401300E8227FBEC07F021C182F40401E7
:1012E000300E8227FBEC07F022C182F40401300E9D
:1012F0008227FBEC07F023C182F40401300E822721
:10130000FBEC07F024C182F40401300E8227FBECD1
:1013100007F025C182F40401300E8227FBEC07F0B0
:1013200026C182F40401300E8227FBEC07F027C1AE
:1013300082F40401300E8227FBEC07F004012C0E2E
:10134000826FFBEC07F00101030E006F000E016FCE
:10135000000E026F000E036F8BEC14F020C182F4BC
:101360000401300E8227FBEC07F021C182F4040156
:10137000300E8227FBEC07F022C182F40401300E0C
:101380008227FBEC07F023C182F40401300E822790
:10139000FBEC07F024C182F40401300E8227FBEC41
:1013A00007F025C182F40401300E8227FBEC07F020
:1013B00026C182F40401300E8227FBEC07F027C11E
:1013C00082F40401300E8227FBEC07F004012C0E9E
:1013D000826FFBEC07F00101180E006F000E016F29
:1013E000000E026F000E036F8BEC14F020C182F42C
:1013F0000401300E8227FBEC07F021C182F40401C6
:10140000300E8227FBEC07F022C182F40401300E7B
:101410008227FBEC07F023C182F40401300E8227FF
:10142000FBEC07F024C182F40401300E8227FBECB0
:1014300007F025C182F40401300E8227FBEC07F08F
:1014400026C182F40401300E8227FBEC07F027C18D
:1014500082F40401300E8227FBEC07F004012C0E0D
:10146000826FFBEC07F0200EF86EF76AF66A040153
:101470000900F5CF82F4FBEC07F00900F5CF82F408
:10148000FBEC07F00900F5CF82F4FBEC07F0090054
:10149000F5CF82F4FBEC07F00900F5CF82F4FBEC0A
:1014A00007F00900F5CF82F4FBEC07F00900F5CF57
:1014B00082F4FBEC07F00900F5CF82F4FBEC07F0B7
:1014C00005EC08F0A6EF0EF08351630AD8A4A6EF4E
:1014D0000EF08451610AD8A4A6EF0EF085516C0A73
:1014E000D8A4A6EF0EF08651410A42E08651440A84
:1014F0001BE08651420AD8B4CBEF0AF08651350A78
:10150000D8B430EF10F08651360AD8B485EF10F019
:101510008651370AD8B4EEEF10F08651380AD8B4A5
:101520004CEF11F0A6EF0EF00798079A04017A0E1F
:10153000826FFBEC07F00401780E826FFBEC07F082
:101540000401640E826FFBEC07F081A8AFEF0AF094
:101550000401550E826FFBEC07F0B4EF0AF00401B2
:101560004C0E826FFBEC07F005EC08F0A6EF0EF0D6
:101570000788079A04017A0E826FFBEC07F00401DA
:10158000410E826FFBEC07F00401610E826FFBECF1
:1015900007F0A5EF0AF00798078A04017A0E826F18
:1015A000FBEC07F00401420E826FFBEC07F0040134
:1015B000610E826FFBEC07F0A5EF0AF0010159679D
:1015C000E9EF0AF05A67E9EF0AF05B67E9EF0AF022
:1015D0005C6701EF0BF04267F5EF0AF04367F5EF48
:1015E0000AF04467F5EF0AF0456701EF0BF00101DF
:1015F000000E006F000E016F000E026F000E036FF1
:1016000012000101620E046F010E056F000E066FDD
:10161000000E076F59C100F15AC101F15BC102F11F
:101620005CC103F1F1EC13F003BF85EF0BF0010196
:10163000000E046FA80E056F550E066F020E076FA1
:1016400059C100F15AC101F15BC102F15CC103F162
:1016500059C179F15AC17AF15BC17BF15CC17CF16E
:10166000F1EC13F003BF3EEF0BF00101000E796FB8
:10167000A80E7A6F550E7B6F020E7C6F0E0E6CEC0F
:1016800006F0E8CF0CF10F0E6CEC06F0E8CF0DF190
:10169000100E6CEC06F0E8CF0EF1110E6CEC06F0BB
:1016A000E8CF0FF13AEC13F079C104F17AC105F1FA
:1016B0007BC106F17CC107F1F1EC13F00782FEEC6F
:1016C00012F03AEC13F00792FEEC12F079C100F13F
:1016D0007AC101F17BC102F17CC103F10792FEECFA
:1016E00012F0CC0E046FE00E056F870E066F050E2C
:1016F000076FF1EC13F000C10CF101C10DF102C153
:101700000EF103C10FF1BDEF0BF00101800E006F70
:101710001A0E016F060E026F000E036F42C104F134
:1017200043C105F144C106F145C107F1F1EC13F0E5
:1017300003AF9EEF0BF0E8EC14F012000E0E6CEC11
:1017400006F0E8CF0CF10F0E6CEC06F0E8CF0DF1CF
:10175000100E6CEC06F0E8CF0EF1110E6CEC06F0FA
:10176000E8CF0FF142C100F143C101F144C102F1E0
:1017700045C103F10782FEEC12F00CC100F10DC16E
:1017800001F10EC102F10FC103F112000401730E49
:10179000826FFBEC07F004012C0E826FFBEC07F06C
:1017A000078455C159F156C15AF157C15BF158C16F
:1017B0005CF13EC142F13FC143F140C144F141C13E
:1017C00045F14AC14CF14BC14DF10794ECEC0BF0E3
:1017D00005EC08F0A6EF0EF059C100F15AC101F175
:1017E0005BC102F15CC103F101018BEC14F0B7ECB9
:1017F00012F00401630E826FFBEC07F004012C0E63
:10180000826FFBEC07F042C100F143C101F144C11A
:1018100002F145C103F101018BEC14F0B7EC12F0B9
:101820000401660E826FFBEC07F004012C0E826F40
:10183000FBEC07F0E8EC14F04CC100F14DC101F1F4
:1018400001018BEC14F0B7EC12F00401740E826FFE
:10185000FBEC07F012000F820401530E826FFBECC9
:1018600007F004012C0E826FFBEC07F083C31EF11E
:1018700084C31FF185C320F186C321F187C322F100
:1018800088C323F189C324F18AC325F18BC326F1D0
:101890008CC327F1010136EC15F0ADEC14F000C15A
:1018A00059F101C15AF102C15BF103C15CF18EC370
:1018B0001EF18FC31FF190C320F191C321F192C398
:1018C00022F193C323F194C324F195C325F196C368
:1018D00026F197C327F1010136EC15F0ADEC14F0B9
:1018E00000C142F101C143F102C144F103C145F11C
:1018F00029EC15F099C323F19AC324F19BC325F178
:101900009CC326F19DC327F1010136EC15F0ADEC27
:1019100014F000C14CF101C14DF1ECEC0BF00401ED
:101920002C0E826FFBEC07F09DEF0CF08251520AF7
:1019300003E10E829DEF0CF00E928251750A03E1D5
:101940000F84A4EF0CF00F948251550A03E10F8627
:10195000ABEF0CF00F9607840FB208EF0DF00FA459
:10196000F4EF0CF0A9C159F1AAC15AF1ABC15BF176
:10197000ACC15CF1ADC15DF1AEC15EF1AFC15FF173
:10198000B0C160F1B1C161F1B2C162F1B3C163F143
:10199000B4C164F1B5C165F1B6C166F1B7C167F113
:1019A000B8C168F1B9C169F1BAC16AF1BBC16BF1E3
:1019B000BCC16CF1BDC16DF1BEC16EF1BFC16FF1B3
:1019C000C0C170F1C1C171F1C2C172F1C3C173F183
:1019D000C4C174F1C5C175F1C6C176F1C7C177F153
:1019E000C8C178F1FCEF0CF055C159F156C15AF15C
:1019F00057C15BF158C15CF13EC142F13FC143F1B7
:101A000040C144F141C145F14AC14CF14BC14DF1D6
:101A100007940EA02AEF0DF00101856717EF0DF076
:101A2000866717EF0DF0876717EF0DF088671BEFDC
:101A30000DF02AEF0DF0DEEC0AF085C104F186C14D
:101A400005F187C106F188C107F1F1EC13F003BF7E
:101A50006EEF0EF0DEEC0AF00101000E046F000ED6
:101A6000056F010E066F000E076F1FEC14F00FA438
:101A700041EF0DF00401750E826FFBEC07F046EFAD
:101A80000DF00401720E826FFBEC07F004012C0EC6
:101A9000826FFBEC07F08BEC14F01D6755EF0DF037
:101AA0000401200E826F58EF0DF004012D0E826F9D
:101AB000FBEC07F024C182F40401300E8227FBEC1A
:101AC00007F025C182F40401300E8227FBEC07F0F9
:101AD00004012E0E826FFBEC07F026C182F4040194
:101AE000300E8227FBEC07F027C182F40401300E90
:101AF0008227FBEC07F004016D0E826FFBEC07F010
:101B000004012C0E826FFBEC07F042C100F143C1CF
:101B100001F144C102F145C103F101018BEC14F064
:101B2000B7EC12F00401480E826FFBEC07F00401E1
:101B30007A0E826FFBEC07F004012C0E826FFBEC37
:101B400007F059C100F15AC101F15BC102F15CC15A
:101B500003F101018BEC14F0B7EC12F00401630EF9
:101B6000826FFBEC07F004012C0E826FFBEC07F098
:101B700059C100F15AC101F15BC102F15CC103F12D
:101B800001010A0E046F000E056F000E066F000EB5
:101B9000076F00EC14F0000E046F120E056F000EBC
:101BA000066F000E076F1FEC14F08BEC14F01EC1D3
:101BB00082F40401300E8227FBEC07F01FC182F48F
:101BC0000401300E8227FBEC07F020C182F40401EF
:101BD000300E8227FBEC07F021C182F40401300EA5
:101BE0008227FBEC07F022C182F40401300E822729
:101BF000FBEC07F023C182F40401300E8227FBECDA
:101C000007F024C182F40401300E8227FBEC07F0B8
:101C100004012E0E826FFBEC07F025C182F4040153
:101C2000300E8227FBEC07F026C182F40401300E4F
:101C30008227FBEC07F027C182F40401300E8227D3
:101C4000FBEC07F00401730E826FFBEC07F004015C
:101C50002C0E826FFBEC07F0E8EC14F04CC100F1A5
:101C60004DC101F1D0EC0FF00EB23AEF0EF00EA024
:101C70006CEF0EF004012C0E826FFBEC07F0200ECF
:101C8000F86EF76AF66A04010900F5CF82F4FBECFE
:101C900007F00900F5CF82F4FBEC07F00900F5CF5F
:101CA00082F4FBEC07F00900F5CF82F4FBEC07F0BF
:101CB0000900F5CF82F4FBEC07F00900F5CF82F4C0
:101CC000FBEC07F00900F5CF82F4FBEC07F009000C
:101CD000F5CF82F4FBEC07F005EC08F00E90A6EFD0
:101CE0000EF00401630E826FFBEC07F004012C0E72
:101CF000826FFBEC07F0ACEC0EF004012C0E826F4F
:101D0000FBEC07F01FEC0FF004012C0E826FFBECD4
:101D100007F09BEC0FF004012C0E826FFBEC07F038
:101D20000101F80E006FCD0E016F660E026F030EFB
:101D3000036FC1EC0EF004012C0E826FFBEC07F078
:101D4000B1EC0FF005EC08F0A6EF0EF00301A26B6A
:101D500007900F92B5EF11F0D8900E0E6CEC06F0D4
:101D6000E8CF00F10F0E6CEC06F0E8CF01F1100E99
:101D70006CEC06F0E8CF02F1110E6CEC06F0E8CF47
:101D800003F10101000E046F000E056F010E066FD6
:101D9000000E076F1FEC14F08BEC14F01EC182F4E0
:101DA0000401300E8227FBEC07F01FC182F404010E
:101DB000300E8227FBEC07F020C182F40401300EC4
:101DC0008227FBEC07F021C182F40401300E822748
:101DD000FBEC07F022C182F40401300E8227FBECF9
:101DE00007F023C182F40401300E8227FBEC07F0D8
:101DF00024C182F40401300E8227FBEC07F025C1D8
:101E000082F40401300E8227FBEC07F004012E0E51
:101E1000826FFBEC07F026C182F40401300E8227AA
:101E2000FBEC07F027C182F40401300E8227FBECA3
:101E300007F004016D0E826FFBEC07F01200120E2A
:101E40006CEC06F0E8CF00F1130E6CEC06F0E8CF76
:101E500001F1140E6CEC06F0E8CF02F1150E6CECFB
:101E600006F0E8CF03F101010A0E046F000E056FC2
:101E7000000E066F000E076F00EC14F0000E046FEA
:101E8000120E056F000E066F000E076F1FEC14F0A8
:101E90008BEC14F01EC182F40401300E8227FBEC9F
:101EA00007F01FC182F40401300E8227FBEC07F01B
:101EB00020C182F40401300E8227FBEC07F021C11F
:101EC00082F40401300E8227FBEC07F022C182F479
:101ED0000401300E8227FBEC07F023C182F40401D9
:101EE000300E8227FBEC07F024C182F40401300E8F
:101EF0008227FBEC07F004012E0E826FFBEC07F04B
:101F000025C182F40401300E8227FBEC07F026C1C4
:101F100082F40401300E8227FBEC07F027C182F423
:101F20000401300E8227FBEC07F00401730E826F70
:101F3000FBEC07F012000A0E6CEC06F0E8CF00F1A3
:101F40000B0E6CEC06F0E8CF01F10C0E6CEC06F019
:101F5000E8CF02F10D0E6CEC06F0E8CF03F1D0EF04
:101F60000FF0060E6CEC06F0E8CF00F1070E6CECFB
:101F700006F0E8CF01F1080E6CEC06F0E8CF02F1B4
:101F8000090E6CEC06F0E8CF03F1D0EF0FF0010181
:101F9000E8EC14F007844AC100F14BC101F1079449
:101FA0000101E80E046F800E056F000E066F000E33
:101FB000076F00EC14F0000E046F040E056F000EA6
:101FC000066F000E076F1FEC14F0880E046F130EDF
:101FD000056F000E066F000E076FF1EC13F00A0E8E
:101FE000046F000E056F000E066F000E076F1FECEA
:101FF00014F08BEC14F001011D6704EF10F00401E4
:10200000200E826F07EF10F004012D0E826FFBECA3
:1020100007F024C182F40401300E8227FBEC07F0A4
:1020200025C182F40401300E8227FBEC07F026C1A3
:1020300082F40401300E8227FBEC07F004012E0E1F
:10204000826FFBEC07F027C182F40401300E822777
:10205000FBEC07F00401430E826FFBEC07F012006B
:1020600087C31EF188C31FF189C320F18AC321F100
:102070008BC322F18CC323F18DC324F18EC325F1D0
:1020800090C326F191C327F101011D6B36EC15F0C9
:10209000ADEC14F00101000E046F000E056F010E8F
:1020A000066F000E076F00EC14F00E0E0C6E00C1F0
:1020B0000BF056EC06F00F0E0C6E01C10BF056EC57
:1020C00006F0100E0C6E02C10BF056EC06F0110E6D
:1020D0000C6E03C10BF056EC06F004017A0E826F11
:1020E000FBEC07F004012C0E826FFBEC07F00401FF
:1020F000350E826FFBEC07F004012C0E826FFBECB7
:1021000007F0ACEC0EF0B4EF0AF087C31EF188C301
:102110001FF189C320F18AC321F18BC322F18CC343
:1021200023F18DC324F18EC325F190C326F191C311
:1021300027F101011D6B36EC15F0ADEC14F0880EA3
:10214000046F130E056F000E066F000E076FF5EC9F
:1021500013F0000E046F040E056F000E066F000EE4
:10216000076F00EC14F00101E80E046F800E056F9C
:10217000000E066F000E076F1FEC14F00A0E0C6EB7
:1021800000C10BF056EC06F00B0E0C6E01C10BF00B
:1021900056EC06F00C0E0C6E02C10BF056EC06F07D
:1021A0000D0E0C6E03C10BF056EC06F004017A0E16
:1021B000826FFBEC07F004012C0E826FFBEC07F042
:1021C0000401360E826FFBEC07F004012C0E826FC7
:1021D000FBEC07F09BEC0FF0B4EF0AF087C31EF1A5
:1021E00088C31FF189C320F18AC321F18BC322F177
:1021F0008CC323F18DC324F18FC325F190C326F145
:1022000091C327F1010136EC15F0ADEC14F0000E8E
:10221000046F120E056F000E066F000E076F00ECC4
:1022200014F001010A0E046F000E056F000E066F18
:10223000000E076F1FEC14F0120E0C6E00C10BF0B5
:1022400056EC06F0130E0C6E01C10BF056EC06F0C6
:10225000140E0C6E02C10BF056EC06F0150E0C6E4F
:1022600003C10BF056EC06F004017A0E826FFBEC12
:1022700007F004012C0E826FFBEC07F00401370E0F
:10228000826FFBEC07F004012C0E826FFBEC07F071
:102290001FEC0FF0B4EF0AF087C31EF188C31FF1E3
:1022A00089C320F18AC321F18BC322F18CC323F1AE
:1022B0008DC324F18EC325F190C326F191C327F17C
:1022C00001011D6B36EC15F0ADEC14F0880E046FB7
:1022D000130E056F000E066F000E076FF5EC13F07E
:1022E000000E046F040E056F000E066F000E076FE0
:1022F00000EC14F00101E80E046F800E056F000E73
:10230000066F000E076F1FEC14F0060E0C6E00C176
:102310000BF056EC06F0070E0C6E01C10BF056ECFC
:1023200006F0080E0C6E02C10BF056EC06F0090E1A
:102330000C6E03C10BF056EC06F004017A0E826FAE
:10234000FBEC07F004012C0E826FFBEC07F004019C
:10235000380E826FFBEC07F004012C0E826FFBEC51
:1023600007F0B1EC0FF0B4EF0AF081A873EF12F0B0
:1023700007A82CEF12F00101800E006F1A0E016FFA
:10238000060E026F000E036F3EC104F13FC105F15E
:1023900040C106F141C107F1F1EC13F003BF73EF47
:1023A00012F0B1EC12F03EC100F13FC101F140C1A9
:1023B00002F141C103F10782FEEC12F00CC104F1FD
:1023C0000DC105F10EC106F10FC107F1F80E006F46
:1023D000CD0E016F660E026F030E036FF1EC13F06A
:1023E0000E0E0C6E00C10BF056EC06F00F0E0C6ECC
:1023F00001C10BF056EC06F0100E0C6E02C10BF092
:1024000056EC06F0110E0C6E03C10BF056EC06F004
:1024100007840101E8EC14F04AC100F14BC101F15D
:1024200007940A0E0C6E00C10BF056EC06F00B0E72
:102430000C6E01C10BF056EC06F00C0E0C6E02C1D6
:102440000BF056EC06F00D0E0C6E03C10BF056ECC3
:1024500006F0079873EF12F007AA73EF12F00784E3
:102460000101E8EC14F04AC100F14BC101F10794FD
:10247000060E0C6E00C10BF056EC06F0070E0C6E4B
:1024800001C10BF056EC06F0080E0C6E02C10BF009
:1024900056EC06F0090E0C6E03C10BF056EC06F07C
:1024A000078455C100F156C101F157C102F158C16D
:1024B00003F10794120E0C6E00C10BF056EC06F0FF
:1024C000130E0C6E01C10BF056EC06F0140E0C6EE0
:1024D00002C10BF056EC06F0150E0C6E03C10BF0AA
:1024E00056EC06F0079A0401805181197F0B0BE02E
:1024F0009EA809D014EE00F081517F0BE126E75031
:10250000812B0F01AD6E71EF07F00CC100F10DC111
:1025100001F10EC102F10FC103F1000E046F000EB4
:10252000056F010E066F000E076F1FEC14F01DA162
:10253000B0EF12F01451D8B4B0EF12F00CC100F1AA
:102540000DC101F10EC102F10FC103F1000E046FC4
:10255000000E056F0A0E066F000E076F1FEC14F0D9
:10256000120001010C6B0D6B0E6B0F6B12001EC184
:1025700082F40401300E8227FBEC07F01FC182F4C5
:102580000401300E8227FBEC07F020C182F4040125
:10259000300E8227FBEC07F021C182F40401300EDB
:1025A0008227FBEC07F022C182F40401300E82275F
:1025B000FBEC07F023C182F40401300E8227FBEC10
:1025C00007F024C182F40401300E8227FBEC07F0EF
:1025D00025C182F40401300E8227FBEC07F026C1EE
:1025E00082F40401300E8227FBEC07F027C182F44D
:1025F0000401300E8227FBEC07F0120001010053AA
:1026000005E1015303E1025301E1002BC1EC13F09A
:10261000E8EC14F02C51006F2D51016F420E046F45
:102620004B0E056F000E066F000E076F00EC14F0E6
:1026300000C104F101C105F102C106F103C107F1B6
:102640000CC100F10DC101F10EC102F10FC103F186
:1026500007B22FEF13F0F5EC13F031EF13F0F1ECBC
:1026600013F000C10CF101C10DF102C10EF103C163
:102670000FF11200E8EC14F04CC100F14DC101F172
:10268000060E6CEC06F0E8CF04F1070E6CEC06F0D9
:10269000E8CF05F1080E6CEC06F0E8CF06F1090E64
:1026A0006CEC06F0E8CF07F1F1EC13F000C118F183
:1026B00001C119F102C11AF103C11BF1290E046F06
:1026C000000E056F000E066F000E076F00EC14F091
:1026D000EE0E046F430E056F000E066F000E076FBF
:1026E000F5EC13F018C104F119C105F11AC106F196
:1026F0001BC107F100EC14F000C110F101C111F190
:1027000002C112F103C113F1120E6CEC06F0E8CF16
:1027100004F1130E6CEC06F0E8CF05F1140E6CEC2E
:1027200006F0E8CF06F1150E6CEC06F0E8CF07F1E5
:102730000D0E006F000E016F000E026F000E036F92
:1027400000EC14F0180E046F000E056F000E066FFB
:10275000000E076F1FEC14F010C104F111C105F158
:1027600012C106F113C107F1F5EC13F06A0E046F04
:102770002A0E056F000E066F000E076FF1EC13F0C6
:102780001200BF0EFA6E200E2D6F2C6BD890003702
:10279000013702370337D8B0D2EF13F02D2FC7EF30
:1027A00013F02C072D070353D8B412000331070B85
:1027B0008009326F03390F0B010F2C6F80EC5FF033
:1027C000336F2C0580EC5FF0335D335F2C6B32335D
:1027D000D8B02C272C3332A9E7EF13F033512C2734
:1027E00012000DEC15F0D8B0120003510719286F34
:1027F000D0EC14F0D8900751031928AF800F1200C5
:10280000286BF4EC14F0D8A00AEC15F0D8B0120044
:10281000DFEC14F0E8EC14F01F0E296F20EC15F03B
:102820000B35D8B0D0EC14F0D8A00335D8B01200D6
:10283000292F0EEF14F028B1F7EC14F01200286BDA
:1028400004510511061107110008D8A0F4EC14F08A
:10285000D8A00AEC15F0D8B01200086B096B0A6B0F
:102860000B6B20EC15F01F0E296F20EC15F00751B3
:102870000B5DD8A448EF14F006510A5DD8A448EFC8
:1028800014F00551095DD8A448EF14F00451085D17
:10289000D8A05BEF14F00451085F0551D8A0053DA6
:1028A000095F0651D8A0063D0A5F0751D8A0073D31
:1028B0000B5FD8900081292F35EF14F028B1F7EC89
:1028C00014F0286BF4EC14F0D89024EC15F00751B8
:1028D0000B5DD8A478EF14F006510A5DD8A478EF08
:1028E00014F00551095DD8A478EF14F00451085D87
:1028F000D8A087EF14F0003F87EF14F0013F87EF77
:1029000014F0023F87EF14F0032BD8B4120028B163
:10291000F7EC14F012000101286BF4EC14F0D8B0BD
:10292000120029EC15F0200E296F0037013702370D
:10293000033711EE27F00A0E2A6FE7360A0EE75C1E
:10294000D8B0E76EE5522A2F9DEF14F0292F95EFAE
:1029500014F028B11D81D890120001010A0E286FD1
:10296000200E296F11EE1DF028512A6F0A0ED89003
:10297000E652D8B0E726E7322A2FB8EF14F0033337
:10298000023301330033292FB2EF14F0E750FF0F69
:10299000D8A00335D8B012001DB1F7EC14F0120026
:1029A000045100270551D8B0053D01270651D8B084
:1029B000063D02270751D8B0073D032712000051FA
:1029C000086F0151096F02510A6F03510B6F12001A
:1029D0000101006B016B026B036B12000101046BC0
:1029E000056B066B076B12000335D8A0120003516C
:1029F000800B001F011F021F031F003F07EF15F090
:102A0000013F07EF15F0023F07EF15F0032B282BCE
:102A1000032512000735D8A012000751800B041FB0
:102A2000051F061F071F043F1DEF15F0053F1DEF93
:102A300015F0063F1DEF15F0072B282B0725120078
:102A40000037013702370337083709370A370B37A2
:102A5000120001011D6B1E6B1F6B206B216B226B23
:102A6000236B246B256B266B276B12001E510F0BFB
:102A70001E6F1F510F0B1F6F20510F0B206F215125
:102A80000F0B216F22510F0B226F23510F0B236F5E
:102A900024510F0B246F25510F0B256F26510F0B5F
:0A2AA000266F27510F0B276F12005D
:10BF0000E844F926000C160C2B0C3F0C520C640C68
:10BF1000760C860C960CA50CB30CC10CCF0CDC0C6B
:06BF2000E80CF40C000C1B
:00000001FF
